:10000000CE29FF3FFF3FFF3F03138312CF03CF03F0
:100010004F08003C03181128CF0300000000000027
:10002000082800000000000008000313831222309B
:10003000DC00D801D901DA01DB01DC0303194B280C
:100040000310DB0CDA0CD90CD80CD30CD20CD10C6D
:10005000D00C031C1D28DC0303193D285408D807C5
:1000600055080318550FD90756080318560FDA0715
:1000700057080318570FDB0721285408D8075508DD
:100080000318550FD90756080318560FDA075708F3
:100090000318570FDB070800073003138312DA0039
:1000A000DA0B50280800031383124908A0008417B4
:1000B0000130D2004A08D1005208D000510803197B
:1000C0006528D00D5010FF3F5F28D00950088005EB
:1000D0004A08A100080003138312C90CC9132008A1
:1000E00084000130CC00CD014D084B02031D7A285D
:1000F0004C084A02031CAD280130D2002108D1006F
:100100005208D000510803198928D00D5010FF3F24
:100110008328500880044908CF0004200130D20011
:100120002108D1005208D000510803199B28D00D96
:100130005010FF3F9528D009500880054908CF008E
:1001400004204D084B06031DA7284A084C06031936
:10015000AD28CC0A0319CD0A74280800E83003132F
:100160008312CB000330CC00CD01CE014908D00072
:100170004A08D100D201D301E830D4000330D500C1
:100180000030D6000030D70015205008CB005108B1
:10019000CC005208CD005308CE0000305302031D9E
:1001A000DB2800305202031DDB2802305102031D00
:1001B000DB28A33050020318DE283529A330D000F5
:1001C0000230D100D201D3014B08D4004C08D50035
:1001D0004D08D6004E08D7005008D4025108031C21
:1001E000510FD5025208031C520FD6025308031CAC
:1001F000530FD7025408CB005508CC005608CD0049
:100200005708CE000530D0005408CB005508CC006C
:100210005608CD005708CE00500803191629CE0CF9
:10022000CD0CCC0CCB0CCE13FF3F0D29FF304B0572
:10023000D8004C08D0005008D8044D08D0004E0813
:10024000D1005008D8044E08D00050085804D400FB
:100250005408003A031935290130CB02031CCC02A3
:10026000031CCD02031CCE0216290800F030031334
:1002700083129F05F03083169F0483129F1749084D
:10028000D000D00D5010D00D501050089F041F14F6
:100290004C209F1400309F180130D2005208013AC0
:1002A000031D542900004A291E08D200D301520818
:1002B000D300D2015208CA005308CB0083161E088F
:1002C0005204CA005308CB000030CB0483121F1025
:1002D0004A08D0004B08D100080003138312DB0149
:1002E000DA01D9018030D800D10CD00C031C81294F
:1002F0005408D90755080318550FDA070318DB0A05
:100300000310D01F89295408DA0755080318550F20
:10031000DB07DB0CDA0CD90CD80C031C74295B0846
:10032000D3005A08D2005908D1005808D00008005C
:1003300003138312D801D9011030DC00510DD80D00
:10034000D90D5408D8025508031C550FD9020318BB
:10035000B0295408D80755080318550FD9070310BA
:10036000D00DD10DDC0B9E29080003138312500819
:10037000D100D0010830DC005108D40C0318C42986
:10038000DC0BBD29D10100340310C929D40C03189A
:10039000D107D10CD00CDC0BC629080007300313A1
:1003A0008312990018308316850018309F008D3015
:1003B00083129F000530C9000530CA005320A201F6
:1003C0006430A300A4013230A5000030A6002C3018
:1003D000A7000130A800BC30A9000230AA00AB0180
:1003E0002B08043C031C192A013085005030C90039
:1003F0002308CA002408CB006B20023085002308A4
:10040000C9002408CA00AE20043085005030C9005D
:100410002308CA002408CB006B2085012308C900EB
:100420002408CA00AE202B08043A0319192AAB0A83
:10043000F0290330C90036215008AC005108AD0046
:10044000A201003085190130D2005208003A031D84
:100450002A2AAB2A02302D02031D302A9E302C029C
:100460000318502A850105140130AB002B08053C08
:10047000031C4F2A093085005030C9002508CA00E6
:100480002608CB006B2085012508C9002608CA0074
:10049000AE202B08053A03194F2AAB0A362A192A2F
:1004A00002302D02031D562ABF302C0203185B2A8E
:1004B00009308500192A02302D02031D612ADF3020
:1004C0002C020318662A0B308500192A02302D02EF
:1004D000031D6C2AFF302C020318712A0D30850091
:1004E000192A03302D02031D772A1F302C0203180E
:1004F0007C2A0C308500192A03302D02031D822A24
:100500003F302C020318872A0E308500192A033049
:100510002D02031D8D2A5F302C020318922A0A3007
:100520008500192A03302D02031D982A7F302C02E2
:1005300003189D2A0F308500192A0F3085002308E3
:10054000C9002408CA00AE2085012308C900240878
:10055000CA00AE20192A2C08D0002D08D100643022
:10056000D400D5016D210630D4005008C5005108D3
:10057000C60054080319C12AC60CC50CC613FF3F98
:10058000BA2A4508AE004608AF002C08D0002D0856
:10059000D1000A30D400D5016D210630D4005008B6
:1005A000BD005108BE0054080319DB2ABE0CBD0C67
:1005B000BE13FF3FD42A3D08B0003E08B1006430AE
:1005C000D400D5013D08D0003E08D1009821500844
:1005D000B2000030D1006430D400D5016D21500844
:1005E000C3005108C4004308B6004408B7004308DC
:1005F000BD02031CBE034408BE020A30D400D5016C
:100600003D08D0003E08D10098215008B3000030CA
:10061000D1000A30D400D5016D215008C100510825
:10062000C2004108B8004208B90041083D02D000AC
:100630004208031C013F3E02D1005008B4000A30BA
:10064000D400B5215008BF003F08BA004308D000CD
:100650004408D1000A30D400D5016D21500845026C
:10066000BD005108031C013F4602BE004108D000F6
:100670004208D1000A30D400D5016D2150083D0256
:10068000D0005108031C013F3E02D1003F08D002B8
:10069000031CD1035008B500AB012B08033C031C1D
:1006A000F72B3230D0002B08500784000008D2000E
:1006B0005208003A031D5F2B3F30BB009E2B5208AF
:1006C000013A031D662B2F30BB009E2B5208023AC5
:1006D000031D6D2B2730BB009E2B5208033A031DD0
:1006E000742B2330BB009E2B5208043A031D7B2B36
:1006F0002130BB009E2B5208053A031D822B20306F
:10070000BB009E2B5208063A031D892B3030BB00DC
:100710009E2B5208073A031D902B3830BB009E2BAE
:100720005208083A031D972B3C30BB009E2B520801
:10073000093A031D9E2B3E30BB009E2BBC013C089A
:10074000073C031CC72B2208013A031DA82BAE2B24
:1007500080303B02031CAD2BCE2BB42B80303B02F0
:10076000031CB32BE12BD12B0130D4003B08D0006C
:1007700054080319BF2BD00D5010FF3FB92B500860
:10078000BB003C08073A0319C72BBC0A9F2BA201E8
:100790002908C9002A08CA00AE20F12B0130A200A6
:1007A000B42B0A3085005030C9002308CA00240841
:1007B000CB006B2085012308C9002408CA00AE20A5
:1007C000B42B0A3085005030C9002708CA00280819
:1007D000CB006B2085012308C9002408CA00AE2085
:1007E000B42B2B08033A0319F72BAB0A4D2B192A0C
:1007F000F82BFF3FFF3FFF3FFF3FFF3FFF3FFF3F24
:02400E00D43F9D
:00000001FF
